:100000000AC01DC01BC01AC019C018C017C016C036
:1000100015C014C013C011271FBFCFE5D0E0DEBF4D
:10002000CDBF20E0A0E4B0E0ECEBF1E402C0319100
:100030003D93A834B207D9F70DD0BEC0E1CF1F93CE
:100040000F930FB70F9310E0F8940F910FBF0F911C
:100050001F911895CF93DF93CDB7DEB7CB50D10B5F
:100060000FB7F894DEBF0FBFCDBF47E0E0E4F0E08C
:10007000AC2FBD2FAF5FBF4F01910D934A95E1F7B4
:1000800041E0C85FDF4F4883C850D04058E0C75FA9
:10009000DF4F5883C950D04052E0C65FDF4F5883CE
:1000A000CA50D04045BB43BB11B94AB7417F4460F9
:1000B0004ABF789481E09BE04AB741604ABF889587
:1000C0004AB74E7F4ABF91B940E050E0A0E0029BA2
:1000D00036C02FE021B9863011F08F5F01C081E07A
:1000E00064E070E031E0E8E0F0E0EC0FFD1FEA0FC3
:1000F000F11FB081B323CF5FDF4F2881C150D040C3
:10010000B227B2B9330F6150710B6117710789F7CC
:1001100061E26A95F1F70000443F21E0520731F4B3
:10012000A23039F0AF5F40E050E006C04F5F5F4F54
:1001300003C040E050E0A0E091B91298C8CF41E57B
:1001400053ECE1E0F0E0EC0FFD1FE80FF11F6FE072
:1001500061B964E070E0B1E0A081AB23CF5FDF4F15
:100160003881C150D040A327A2B9BB0F6150710B99
:100170006117710789F721E22A95F1F7000091B91B
:100180001298029905C04150510B41175107F9F6D9
:10019000029B0FC04FE041B9CF5FDF4F4881C15094
:1001A000D04042B961E26A95F1F7000091B9129826
:0C01B000EFCF11B9789480CFF894FFCF06
:0801BC000B04010503070B0011
:00000001FF
